:100000000C9483060C94951D0C946E1D0C94AB06F9
:100010000C94AB060C94611F0C94AB060C94331F2C
:100020000C94A61F0C94AB060C94AB060C94AB0678
:100030000C94AB060C94AB060C94AB060C94AB067C
:100040000C94241D0C94AB060C94E21D0C94BC1D66
:100050000C94AB060C94AB060C94AB060C94AB065C
:100060000C94141E0C94AB06680318017268188077
:10007000234020034C69676874734F4E04034F4E4E
:10008000042020202020BE5004B03B805F50046834
:100090003B0205680576380A01285004683B282F82
:1000A0006805183802004F680576380A00295004A0
:1000B000683B212650046832101E50046832111F1C
:1000C000C004BF1103696804800200EE8003680168
:1000D000EA1804FF0200E16804C00200AEC0036831
:1000E00001AA681880234020035354414E444259CA
:1000F0002004032020042020202020E468188023EE
:100100004020032041555820492F5004032020044B
:100110002020202020E968188023402003432E203F
:10012000446973632004032020042020202020C37E
:1001300068188023402003425420417564696F048D
:10014000032020042020202020F368188023402052
:1001500003555342617564696F0403202004202015
:10016000202020A168188023402003464D20426EA5
:1001700064203304032020042020202020E368187A
:100180008023402003464D20626E64203204032009
:1001900020042020202020C268188023402003460D
:1001A0004D20626E64203104032020042020202092
:1001B00020C16818802340200344414220626E64BD
:1001C0003104032020042020202020AD6818802343
:1001D000402003414D20426E64203104032020045E
:1001E0002020202020E6681880234020034441423C
:1001F00020626E643304032020042020202020AFDE
:100200006818802340200344414220626E64320417
:10021000032020042020202020AE68051838030089
:100220004E68057638030020180A68390209003F35
:10023000000101776805183801004C00000000003B
:100240003E5B4F5B3E3E6B4F6B3E1C3E7C3E1C1844
:100250003C7E3C181C577D571C1C5E7F5E1C0018A2
:100260003C1800FFE7C3E7FF0018241800FFE7DB96
:10027000E7FF30483A060E2629792926407F0505F2
:1002800007407F05253F5A3CE73C5A7F3E1C1C082F
:10029000081C1C3E7F14227F22145F5F005F5F06F4
:1002A000097F017F006689956A606060606094A242
:1002B000FFA29408047E040810207E201008082A5B
:1002C0001C08081C2A08081E101010100C1E0C1EFA
:1002D0000C30383E3830060E3E0E0600000000009E
:1002E00000005F00000007000700147F147F142443
:1002F0002A7F2A12231308646236495620500008C8
:10030000070300001C2241000041221C002A1C7F20
:100310001C2A08083E0808008070300008080808F9
:1003200008000060600020100804023E5149453E6C
:1003300000427F400072494949462141494D3318E6
:1003400014127F1027454545393C4A49493141211E
:100350001109073649494936464949291E00001402
:10036000000000403400000008142241141414144A
:1003700014004122140802015909063E415D594EFC
:100380007C1211127C7F494949363E414141227F0E
:100390004141413E7F494949417F090909013E41A7
:1003A0004151737F0808087F00417F410020404190
:1003B0003F017F081422417F404040407F021C02E1
:1003C0007F7F0408107F3E4141413E7F09090906B5
:1003D0003E4151215E7F0919294626494949320388
:1003E000017F01033F4040403F1F2040201F3F400E
:1003F00038403F63140814630304780403615949C7
:100400004D43007F41414102040810200041414119
:100410007F040201020440404040400003070800FE
:1004200020545478407F2844443838444444283881
:100430004444287F385454541800087E090218A4F4
:10044000A49C787F0804047800447D40002040404C
:100450003D007F1028440000417F40007C04780468
:10046000787C080404783844444438FC1824241860
:1004700018242418FC7C0804040848545454240408
:10048000043F44243C4040207C1C2040201C3C4035
:1004900030403C44281028444C9090907C44645454
:1004A0004C44000836410000007700000041360847
:1004B0000002010204023C2623263C1EA1A1611277
:1004C0003A4040207A3854545559215555794122A3
:1004D00054547842215554784020545579400C1E8C
:1004E0005272123955555559395454545939555435
:1004F00054580000457C410002457D420001457C86
:10050000407D1211127DF0282528F07C54554500BD
:100510002054547C547C0A097F4932494949323A73
:100520004444443A324A4848303A4141217A3A42B6
:10053000402078009DA0A07D3D4242423D3D40408C
:10054000403D3C24FF2424487E4943662B2FFC2F4A
:100550002BFF0929F620C0887E09032054547941D5
:100560000000447D413048484A32384040227A00F9
:100570007A0A0A727D0D19317D2629292F2826290C
:1005800029292630484D402038080808080808085E
:1005900008382F10C8ACBA2F102834FA00007B009E
:1005A0000008142A142222142A1408550055005554
:1005B000AA55AA55AAFF55FF55FF000000FF0010DD
:1005C0001010FF00141414FF001010FF00FF101093
:1005D000F010F0141414FC001414F700FF0000FFD6
:1005E00000FF1414F404FC141417101F10101F1033
:1005F0001F1414141F00101010F0000000001F1032
:100600001010101F10101010F010000000FF10103C
:1006100010101010101010FF10000000FF14000048
:10062000FF00FF00001F10170000FC04F414141753
:1006300010171414F404F40000FF00F71414141439
:10064000141414F700F7141414171410101F101FAB
:10065000141414F4141010F010F000001F101F00F8
:1006600000001F14000000FC140000F010F0101037
:10067000FF10FF141414FF141010101F00000000CE
:10068000F010FFFFFFFFFFF0F0F0F0F0FFFFFF00C2
:1006900000000000FFFF0F0F0F0F0F3844443844D5
:1006A000FC4A4A4A347E02020606027E027E026349
:1006B000554941633844443C04407E201E200602D4
:1006C0007E020299A5E7A5991C2A492A1C4C7201B1
:1006D000724C304A4D4D303048784830BC625A46F2
:1006E0003D3E494949007E0101017E2A2A2A2A2AE3
:1006F00044445F444440514A444040444A514000CD
:1007000000FF0103E080FF000008086B6B08361251
:10071000362436060F090F060000181800000010D6
:1007200010003040FF0101001F01011E00191D17BC
:1007300012003C3C3C3C0000000000000103070F9D
:100740001F3F7F0080C0E0F0F8FCFEDB40A4A62E37
:10075000AF2000A1C8D300408DAED580A8000060B6
:100760000000000000000000000000000000E000A9
:1007700000000000000000000000000001E0000098
:10078000000000000000000000000001F000000078
:100790000000000000000000000003F00000000066
:1007A00000000000000000000007F0000000000052
:1007B000000000000000000007F80000000000003A
:1007C000000000000000000FF800000003C0007EE1
:1007D000000001E0007F0FF800000003C000FE00F1
:1007E0000001E000FFEFF800000003C000FE000081
:1007F00001E000FFFFF800000003C000F00000006F
:100800000F007FFE7FC0000003C000F00000000F5B
:10081000003FFE7FF83FF1FBCFFCFEF3BC3DEFE075
:100820001FFE7FFF7FFBFFDFFEFEFFBC3DEFE01FF3
:10083000C6FFFF7FFBFFDFFEFEFFBC3DEFE00FE3E7
:10084000C7FE787BC3DE1EF0FFBC3DEF0007FF87CD
:10085000FC787BC3DE1EF0F83C3DEF0001FFFFF0AB
:10086000007BC3C01EF0F03C3DEF0001F37FE03F92
:10087000FBC3CFFEF0F03C3DEF0003E33F807FFB86
:10088000C3DFFEF0F03C3DEF0007E73C00787BC3A0
:10089000DE1EF0F03C3DEF0007FFBE00787BC3DEBC
:1008A0001EF0F03C3DEF0007FFFE00787BC3DE1E2C
:1008B000F0F03C3DEF000FFFFE007FFBFFDFFEF09E
:1008C000F03FFDEFE00FFFFF007FFBFFDFFEF0F0EA
:1008D0003FFDEFE00FF9FF003E79F9CF9EF0F01FEA
:1008E0003DE7E01FF1FF00000000000000000000F5
:1008F00000001F80FF007FFFFFFFFFFFFFFFFFFFE4
:10090000E01C007F007FFFFFFFFEB46D888D18E0C4
:1009100000001F007FFFFFFFFE95AD7DB577E00073
:10092000000F007FFFFFFFFEA5AD9D8D19E00000C9
:1009300006007FFFFFFFFEB5ADEDB57EE0000000D5
:1009400000000180000000000000000000038000A3
:10095000000000000000000007C0000000000000D0
:1009600000000007C00000000000000000000FC0F1
:100970000000000000000000001FE0000000000078
:10098000000000001FE00000000000000000003F29
:10099000E00000000000000000003FF00000000048
:1009A00000000000007FF0000000000000001FF8C1
:1009B0007FF0000000000000003FFE7FF00000001C
:1009C000000000003FFF7FF0000000000000001F5B
:1009D000FFFBE0000000000000000FFFF9FFC00077
:1009E00000000000000FFFF9FFF800000000000009
:1009F00007FFF1FFFF00000000000003FC73FFFF92
:100A000080000000000001FE3FFFFF8000000000AA
:100A10000000FF1E0FFF000000000000007FFE1F0F
:100A2000FC000000000000003FFFFFF80000000095
:100A30000000000FDFFFE0000000000000001F19B1
:100A4000FFC0000000000000003F3CFF000000006D
:100A5000000000007E7CF800000000000000007F25
:100A6000FE7C0000000000000000FFFFFC00000012
:100A70000000000000FFFFFE00000000000000007A
:100A8000FFFFFE0000000000000001FFEFFE00007D
:100A9000000000000001FFCFFE0000000000000089
:100AA00003FF07FE0000000000000003FC07FE003B
:100AB00000000000000003F003FE00000000000042
:100AC00000018000FE000000000000000000007E29
:100AD000000000000000000000003E0000000000D8
:100AE00000000000000C000000000000078000FC77
:100AF000000003C0000000078001FC000003C000EC
:100B00000000078001FC000003C000000007800116
:100B1000E00000001E000000078001E00000001E51
:100B2000007FE3F79FF9FDE7787BDFC0FFF7FFBFAA
:100B3000FDFDFF787BDFC0FFF7FFBFFDFDFF787B8A
:100B4000DFC0F0F787BC3DE1FF787BDE00F0F78780
:100B5000BC3DE1F0787BDE0000F787803DE1E07886
:100B60007BDE007FF7879FFDE1E0787BDE00FFF70B
:100B700087BFFDE1E0787BDE00F0F787BC3DE1E078
:100B8000787BDE00F0F787BC3DE1E0787BDE00F0AB
:100B9000F787BC3DE1E0787BDE00FFF7FFBFFDE1BA
:100BA000E07FFBDFC0FFF7FFBFFDE1E07FFBDFC0C1
:100BB0007CF3F39F3DE1E03E7BCFC00000000000EE
:100BC000000000000000FFFFFFFFFFFFFFFFFFFF2F
:100BD000C0FFFFFFFFFD68DB111A31C0FFFFFFFF01
:100BE000FD2B5AFB6AEFC0FFFFFFFFFD4B5B3B1A7B
:100BF00033C0FFFFFFFFFD6B5BDB6AFDC057616920
:100C000074696E6720666F7220492D4275730053B8
:100C1000706565642F52504D206D6F6E69746F72F0
:100C2000004E4558542054455354005353443133D7
:100C3000303620616C6C6F636174696F6E20666121
:100C4000696C65640052504D3A2000206B6D2F682E
:100C5000004D65747269633A200020204163747509
:100C6000616C3A2000202053796E6320553A2000B1
:100C7000202053796E6320443A200020204175746F
:100C80006F3A204F4646005461726765743A2000FF
:100C9000204D50480053706565643A20006804BFD9
:100CA0000201D000000000240027002A00000000FC
:100CB00000250028002B00000000080002010000B1
:100CC00003040700000000000000002200FF2100D4
:100CD0000000002300260029000404040404040486
:100CE00004020202020202030303030303010204DB
:100CF000081020408001020408102001020408109E
:100D000020008920552011241FBECFEFD8E0DEBF80
:100D1000CDBF25E0A2EAB1E001C01D92A633B20723
:100D2000E1F711E0A0E0B1E0E8EBF5E502C00590E5
:100D30000D92A23AB107D9F716E0C2E8D6E004C096
:100D40002197FE010E948F29C138D107C9F70E945F
:100D5000B3210C94CF2A0C9400000895833081F0C5
:100D600028F4813099F08230A9F008958730A9F0F5
:100D70008830C9F08430B1F4809180008F7D03C049
:100D8000809180008F7780938000089584B58F775D
:100D900084BD089584B58F7DFBCF8091B0008F779F
:100DA0008093B00008958091B0008F7DF9CFCF93EC
:100DB000DF93282F30E0F901E954F34F8491F901D2
:100DC000E351F34FD491F901E752F34FC491CC238F
:100DD000A1F081110E94AE06EC2FF0E0EE0FFF1F94
:100DE000E153F34FA591B491EC91ED2381E090E0B4
:100DF00009F480E0DF91CF91089580E090E0FACF90
:100E00001F93CF93DF93282F30E0F901E954F34F7C
:100E10008491F901E351F34FD491F901E752F34F73
:100E2000C491CC23A9F0162F81110E94AE06EC2F9D
:100E3000F0E0EE0FFF1FE355F34FA591B4918FB78C
:100E4000F894EC91111108C0D095DE23DC938FBF8C
:100E5000DF91CF911F910895DE2BF8CFCF93DF93D1
:100E600090E0FC01E351F34F24918752934FFC0132
:100E700084918823C9F090E0880F991FFC01ED55FB
:100E8000F34FA591B491FC01E355F34FC591D49173
:100E900061110DC09FB7F8948C91209582238C939B
:100EA0008881282328839FBFDF91CF9108956230E6
:100EB00051F49FB7F8943C91822F809583238C93B3
:100EC000E8812E2BEFCF8FB7F894EC912E2B2C933B
:100ED0008FBFEACF3FB7F894809181029091820250
:100EE000A0918302B091840226B5A89B05C02F3F34
:100EF00019F00196A11DB11D3FBFBA2FA92F982F40
:100F00008827BC01CD01620F711D811D911D42E03A
:100F1000660F771F881F991F4A95D1F708958F9202
:100F20009F92AF92BF92CF92DF92EF92FF924B01CE
:100F30005C010E946A076B017C010E946A076C19C0
:100F40007D098E099F09683E734081059105A8F3CC
:100F500021E0821A9108A108B10888EEC80E83E04A
:100F6000D81EE11CF11C81149104A104B10429F7DD
:100F7000FF90EF90DF90CF90BF90AF909F908F90B9
:100F800008952FB7F89460917D0270917E02809150
:100F90007F02909180022FBF0895089508950895CB
:100FA0000895EF92FF920F931F93CF93DF938C01DD
:100FB0007B01D0E0C0E0F701EC0FFD1F64916623D8
:100FC00061F0D801ED91FC910190F081E02DC80114
:100FD0000995892B11F02196EECFCE01DF91CF91AB
:100FE0001F910F91FF90EF900895AF92BF92CF9213
:100FF000DF92EF92FF920F931F93CF93DF936C01D9
:101000007B018B01040F151FEB015E01AE18BF08B9
:10101000C017D10759F06991D601ED91FC9101906B
:10102000F081E02DC6010995892B79F7C501DF9183
:10103000CF911F910F91FF90EF90DF90CF90BF90D5
:10104000AF900895FC01538D448D252F30E0842FFF
:1010500090E0821B930B541710F0CF9608950197E0
:101060000895FC01918D828D981761F0A28DAE0FCD
:10107000BF2FB11D5D968C91928D9F5F9F73928F54
:1010800090E008958FEF9FEF0895FC01918D828D80
:10109000981731F0828DE80FF11D858D90E008954D
:1010A0008FEF9FEF0895FC01918D228D892F90E0A5
:1010B000805C9F4F821B91098F739927089589E85F
:1010C00092E00E94530821E0892B09F420E0822F4E
:1010D000089580E090E0892B29F00E945F0881113B
:1010E0000C9400000895FC01A48DA80FB92FB11D28
:1010F000A35ABF4F2C91848D90E001968F7399274E
:10110000848FA689B7892C93A089B1898C9183702B
:1011100080648C93938D848D981306C00288F38924
:10112000E02D80818F7D80830895EF92FF920F9351
:101130001F93CF93DF93EC0181E0888F9B8D8C8D83
:1011400098131AC0E889F989808185FF15C09FB777
:10115000F894EE89FF896083E889F989808183703A
:10116000806480839FBF81E090E0DF91CF911F91E9
:101170000F91FF90EF900895F62E0B8D10E00F5F0A
:101180001F4F0F731127E02E8C8D8E110CC00FB6E0
:1011900007FCFACFE889F989808185FFF5CFCE0178
:1011A0000E947308F1CFEB8DEC0FFD2FF11DE35A78
:1011B000FF4FF0829FB7F8940B8FEA89FB898081FB
:1011C0008062CFCFCF93DF93EC01888D8823B9F075
:1011D000AA89BB89E889F9898C9185FD03C0808142
:1011E00086FD0DC00FB607FCF7CF8C9185FFF2CFBF
:1011F000808185FFEDCFCE010E947308E9CFDF919A
:10120000CF910895EF92FF920F931F93CF93DF93A7
:10121000EC01EC80FD806E157F050CF070C057FF6F
:1012200004C0240F351F50E040E08E819F81FA01F9
:10123000E20FF31F8E179F071CF49C01241B350B34
:10124000121613060CF05BC0922F842F869586959C
:1012500086958E9DD0018F9DB00D11246A0F7B1F46
:10126000AF8DB8A1A60FB71F477049F188E0841B66
:10127000482F682F70E0FB01ED5BF84FE4912817D1
:1012800008F063C0621B71092FEF30E002C0359592
:1012900027956A95E2F7E2230130110539F0B0F1A4
:1012A0000230110561F58C91E82702C08C91E82B82
:1012B000EC93941720F12C813D81A20FB31FE92FED
:1012C000E41BE83078F00230110521F58E2F9C9157
:1012D00090959C932C813D81A20FB31F885088303C
:1012E000B0F7E770EE2359F0F0E0E55CF84FE491D9
:1012F00001301105F9F010F10230110519F1DF91FB
:10130000CF911F910F91FF90EF900895E0958C91F0
:10131000E823CECF81E00115110509F480E0819525
:101320009E2F8C932C813D81A20FB31F9850983033
:10133000C0F7D7CF8C91E82BEC93E1CFE0958C915F
:10134000E823FACF8C91E827F7CF0130110509F493
:10135000ADCFE0F20230110509F4A5CFAE0DBF1DEF
:10136000AECF0F931F93CF93DF9377FF04C0260F69
:10137000371F70E060E0DC011496CD91DC91FB0139
:10138000E20FF31FCE17DF071CF49E01261B370B5D
:10139000121613064CF5FA0157FD3796A3E0F595A2
:1013A000E795AA95E1F7EC9FD001ED9FB00DFC9F6A
:1013B000B00D11246A0F7B1FDC015F96ED91FC914B
:1013C000E60FF71F4770552781E090E001C0880FB6
:1013D0004A95EAF7482F0130110559F0A8F02E0F71
:1013E0003F1F02301105E1F0DF91CF911F910F9166
:1013F00008952E0F3F1FE217F307B1F38191DF012C
:101400001197842B8C93F7CF80952E0F3F1FE217F7
:10141000F30751F39191DF01119798239C93F7CF34
:10142000E217F30709F38191DF01119784278C9369
:10143000F7CF0F931F93FA01DC0156964C91569704
:101440004230E9F04330A1F1413061F514964D91FD
:101450005C91DA01AE1BBF0BFD01E21BF30B77FDC4
:101460000BC0DC0116964D915C916417750724F44E
:10147000AB01BF010E94B1091F910F91089514960D
:101480004D915C91DA01A61BB70BBD01615071094A
:10149000DC0116964D915C91DA01AE1BBF0BFD018C
:1014A000E21BF30B77FDE8CFAF010E940209E4CF06
:1014B00016964D915C91DA01A61BB70BBD016150E8
:1014C0007109CDCF0F931F93FA01DC0156964C9111
:1014D00056974230A9F0433091F1413019F51496F6
:1014E0004D915C91DA01AE1BBF0BFD013197F7FD09
:1014F00004C0AB01BF010E9402091F910F91089522
:1015000014964D915C91DA01A61BB70BBD01DC016D
:1015100016964D915C91DA01AE1BBF0BFD01319720
:10152000621B730BF7FDE9CFDC0116964D915C91C0
:10153000E417F50714F7AF010E94B109DECF169644
:101540004D915C91DA01A61BB70BBD01621B730BB9
:10155000CECFFC0177FD64C080859185681779073F
:101560000CF05EC057FD5CC0828593854817590713
:101570000CF056C086898230B1F0833029F1813079
:1015800041F484819581841B950BAB01BC016150B2
:1015900071092130310509F108F443C022303105C9
:1015A00009F463C0089584819581DC01A61BB70B03
:1015B000BD016150710986819781DC01A41BB50BC7
:1015C000AD0141505109E5CF86819781861B970B6C
:1015D000BA01AC0141505109DCCFCA0157FD079651
:1015E000A3E095958795AA95E1F7A481B5818A9F97
:1015F00090018B9F300D9A9F300D1124620F731F45
:10160000078CF0A1E02DE60FF71F4770552721E06A
:1016100030E001C0220F4A95EAF78081822B808357
:101620000895CA0157FD079633E0959587953A9539
:10163000E1F7A481B5818A9F90018B9F300D9A9F1D
:10164000300D1124620F731F078CF0A1E02DE60FFF
:10165000F71F4770552781E090E001C0880F4A9539
:10166000EAF7809590818923DACFCA0157FD079662
:1016700023E0959587952A95E1F7A481B5818A9F06
:1016800090018B9F300D9A9F300D1124620F731FB4
:10169000078CF0A1E02DE60FF71F4770552721E0DA
:1016A00030E001C0220F4A95EAF780818227B7CF48
:1016B00008958EBD00000DB407FEFDCF8EB50895D0
:1016C0008CBD9DBD08950895FC016370668B848177
:1016D000958126813781613039F0633029F0918717
:1016E0008087338722870895318720879387828771
:1016F00008952F923F924F925F926F927F928F92B6
:101700009F92AF92BF92CF92DF92EF92FF920F9390
:101710001F93CF93DF93CDB7DEB76A970FB6F894D8
:10172000DEBF0FBECDBF9A8F898F7A8369834A014E
:10173000D22E18870F833701BC2CDC0159962D91CE
:101740003C915A972115310509F015C118968D91D4
:101750009C911997681779070CF0D7C11A968D914B
:101760009C91481759070CF0D0C14C2C512CB6E075
:10177000CB9E600D711D11247C876B871616170692
:101780000CF0C3C1EA2DF0E0FA87E98793E0EE0F91
:10179000FF1F9A95E1F7F88BEF87CF01840F951F14
:1017A000181619060CF0B1C1A98DBA8D58968C91F6
:1017B000811104C0BFEABD1508F4D394A98DBA8D78
:1017C000ED91FC9111970284F385E02DCD010995EF
:1017D000B5E0DB9EC0011124E981FA81FC83EB8333
:1017E000312C212C9C01255C3D4F388F2F8B4A2DAD
:1017F00050E05E8B4D8BEF89F88DE20DF31D449127
:101800009E828D82D12CC12C69817A81620D731DDB
:101810007A8B698B842F90E09C8B8B8BE98DFA8D72
:10182000A081B18140FF82C0F1E0BF126FC0AF1252
:101830006DC01C96ED91FC912F813885A4014C0D53
:101840005D1D69897A89898D9A8D0995EB89FC8955
:10185000F595E7954E2F5FEFC51AD50A6D817E810C
:101860008D899E89680F791F7E836D8398E0C916E4
:10187000D10481F6AFEF2A1A3A0AEB81FC81E40D1C
:10188000F51DFC83EB83F5E02F16310409F0B3CF8F
:101890002F81388526153705B9F0A98DBA8DED91C0
:1018A000FC91B1E0BB1257C0AB1255C069817A817F
:1018B0006B5F7F4F0088F189E02D830128E030E0E5
:1018C000A401898D9A8D0995A98DBA8DED91FC9110
:1018D00011970688F789E02DCD016A960FB6F89426
:1018E000DEBF0FBECDBFDF91CF911F910F91FF9053
:1018F000EF90DF90CF90BF90AF909F908F907F90B0
:101900006F905F904F903F902F9009941E96ED91AD
:10191000FC91EF80F88409851A8592014D815E81E2
:101920006B817C81898D9A8D099590CF2F81388527
:101930002615370509F48ACF31E0B31207C0A31288
:1019400005C01C96ED91FC91930178CF1E96ED9108
:10195000FC917301E0CF6B857C8564197509068461
:10196000F785E02D73010F8518899201A401898DF7
:101970009A8D0995A9CFF9013496949132974591A2
:101980005491D91AB7E0DB9E400D511D1124F90185
:10199000259134913C8B2B8BFA0125903490FA01E0
:1019A0003296749031963491398B32966490319698
:1019B000449041E04C1518F04A1508F07FC0662DA0
:1019C000062C000C770B7C836B83842D042C000C7D
:1019D000990B9E838D83A98DBA8DED91FC91119702
:1019E0000284F385E02DCD010995512CD12CC12C19
:1019F000EA2DF0E0FA87E9872B2D30E03C872B8732
:101A0000A401440D511D47FC5A95588F4F8B698195
:101A10007A81660D711D67FC7A957E876D8779895D
:101A2000C71608F051CF2C2D30E04D815E81420F5A
:101A3000531FA985BA854A9FC0014B9F900D5A9F9D
:101A4000900D1124FC01E80DF91DF88BEF87852D11
:101A5000612C4F89588D420F531F5E8B4D8B67143D
:101A600008F050C044244394480E877041F4C101EB
:101A70000196EB89FC89E20DF31DD4901C01D7FE81
:101A800019C0A98DBA8DED91FC91662D70E0B1E081
:101A9000BB1219C0AB1217C02D853E85620F731F94
:101AA0000484F585E02D2F8138854D895E89898DE7
:101AB0009A8D0995DD0C6394842DD1CF1E821D82F1
:101AC0001C821B8288CF4B815C81640F751FAB85A4
:101AD000BC856A9FC0016B9F900D7A9F900D112469
:101AE00069817A81680F791F0684F785E02DEF8080
:101AF000F88409851A859D014F855889898D9A8DAD
:101B00000995D8CF570CC3948ACF6A960FB6F8942C
:101B1000DEBF0FBECDBFDF91CF911F910F91FF9020
:101B2000EF90DF90CF90BF90AF909F908F907F907D
:101B30006F905F904F903F902F9008958F929F925B
:101B4000AF92CF92EF92FF920F931F93CF93DF93B9
:101B5000EC01262F898D9A8D009709F051C06A30CB
:101B6000D1F41D861C868D8948E0849F9001112444
:101B70008E859F85820F931F9F878E8781E090E0DF
:101B8000DF91CF911F910F91FF90EF90CF90AF9089
:101B90009F908F9008956D3089F3CC88AD888F89A0
:101BA0008823C1F08C859D8536E0C39E800D911DF4
:101BB0001124488559854817590764F44E855F8577
:101BC0001D861C8638E0A39EC0011124840F951F3A
:101BD0009F878E87EA88FB88088919894E855F85EB
:101BE0006C857D85CE010E94790B2C898C859D8525
:101BF00046E0249F800D911D11249D878C87BECFC8
:101C00006A3069F41D861C86FC013896E4912D89A2
:101C10008E859F85E29F800D911D1124ADCF6D3083
:101C200009F4ACCFFC0134963491631708F4A6CFC5
:101C30003296E491E61708F4A1CFFC013296859024
:101C40009490462F431B342F47E0349F800C911C07
:101C50001124F401329634913196E4913323A9F1A1
:101C6000EE2399F1CC88F4013596E491AD884F8943
:101C7000442301F10E2E000CFF0BE30FF11DCE9E4D
:101C8000A001CF9E500D11246C857D85460F571FF6
:101C900068857985641775076CF44E855F851D86A8
:101CA0001C86FC013896E491AE9E400D511D112416
:101CB0005F874E87EA88FB88088919894E855F858A
:101CC0006C857D85CE010E94790BF4013496E491F8
:101CD0002C898C859D85E29F800D911D11248DCFCF
:101CE0006F927F928F929F92AF92BF92CF92DF922C
:101CF000EF92FF920F931F93CF93DF93EC016B0151
:101D00005A0139014801E881F9810284F385E02D07
:101D10000995E881F9810288F389E02D8701930113
:101D2000A501B601CE010995A501480D591D4150E7
:101D30005109E881F9810288F389E02D9301B60108
:101D4000CE010995E881F9810088F189E02D94019F
:101D5000A501B601CE010995C60CD71CB60161508C
:101D60007109E881F9810088F189E02D9401A501CC
:101D7000CE010995E881F9810688F789E02DCE0129
:101D8000DF91CF911F910F91FF90EF90DF90CF9057
:101D9000BF90AF909F908F907F906F9009946F92BB
:101DA0007F928F929F92AF92BF92CF92DF92EF92EB
:101DB000FF920F931F93CF93DF935C01EB016A01B6
:101DC000490138018701DC01ED91FC91621773072D
:101DD00019F5641675062CF0962D872D3A01C92E3B
:101DE000D82E9601261937092F5F3F4F048CF58DA9
:101DF000E02DA301BE01C5010995DF91CF911F918F
:101E00000F91FF90EF90DF90CF90BF90AF909F9099
:101E10008F907F906F9008954615570591F426177F
:101E2000370724F0892D4B01C22FD82F9E01281986
:101E300039092F5F3F4F068CF78DE02DA601B401C5
:101E4000DACF0284F385E02D0995D501ED91FC915F
:101E50000488F589E02D83019401A601BE01C50126
:101E60000995D501ED91FC910688F789E02DC50112
:101E7000DF91CF911F910F91FF90EF90DF90CF9066
:101E8000BF90AF909F908F907F906F900994EF924A
:101E9000FF920F931F93DC011A960D911C911B97D3
:101EA00018962D913C911997ED91FC9100A0F1A10C
:101EB000E02D7B0150E040E070E060E009951F916B
:101EC0000F91FF90EF9008954F925F926F927F92E3
:101ED0008F929F92AF92BF92CF92DF92EF92FF923A
:101EE0000F931F93CF93DF936C012B015A0139019C
:101EF0004801DC01ED91FC910284F385E02D099508
:101F0000E201640C751CD601ED91FC91C615D70554
:101F10005CF40088F189E02D87019401A501BE01E0
:101F2000C60109952196EFCF0688F789E02DC601F5
:101F3000DF91CF911F910F91FF90EF90DF90CF90A5
:101F4000BF90AF909F908F907F906F905F904F90D9
:101F500009948F929F92AF92BF92CF92DF92EF92AD
:101F6000FF920F931F93CF93DF93EC015B014A0124
:101F70006901E881F9810284F385E02D09959501D5
:101F80002C0D3D1D21503109E881F9810488F58926
:101F9000E02D78018401A401B501CE010995E88105
:101FA000F9810688F789E02DCE01DF91CF911F914D
:101FB0000F91FF90EF90DF90CF90BF90AF909F90E8
:101FC0008F9009948F929F92AF92BF92CF92DF929F
:101FD000EF92FF920F931F93CF93DF93EC015B017E
:101FE0004A0169017801E881F9810284F385E02DD5
:101FF0000995C80CD91C860101501109E881F981A5
:102000000488F589E02D9501A401B501CE0109955B
:10201000E881F9810688F789E02DCE01DF91CF9123
:102020001F910F91FF90EF90DF90CF90BF90AF90F6
:102030009F908F900994EF92FF920F931F93DC0172
:10204000ED91FC9100A0F1A1E02D09951F910F9158
:10205000FF90EF9008950F931F93DC01ED91FC9199
:10206000068CF78DE02D09951F910F9108950F9320
:102070001F93DC01ED91FC91048CF58DE02D099509
:102080001F910F910895DC01ED91FC910084F18581
:10209000E02D09943F924F925F926F927F928F92C0
:1020A0009F92AF92BF92CF92DF92EF92FF920F93E7
:1020B0001F93CF93DF935C017B014A0169013901D2
:1020C00087E0680E711C93E0759467949A95E1F728
:1020D0002B01400E511E10E000E0312CD0E0C0E09A
:1020E000CE0187709927330C892B59F4FE0183E0C8
:1020F000F595E7958A95E1F7E00FF11FE80DF91DD9
:10210000349037FE0AC021E030E0A701B5016C0F22
:102110007D1F8AED94E00E9443102196CC16DD06C7
:10212000F9F68FEFE81AF80A060D171DE414F50406
:10213000A9F6DF91CF911F910F91FF90EF90DF9063
:10214000CF90BF90AF909F908F907F906F905F9057
:102150004F903F9008952F923F924F925F926F92CF
:102160007F928F929F92AF92BF92CF92DF92EF9227
:10217000FF920F931F93CF93DF9300D000D000D036
:10218000CDB7DEB73C016A013E832D83FC82EB8232
:102190005801A41AB50AB7FE03C0B194A194B108BE
:1021A0008D809E80861A970A97FE03C09194819431
:1021B00091088A149B045CF0902F812F0D811E8161
:1021C0009D838E839C2D8D2D6B01692F782F0C158F
:1021D0001D055CF09D818E817E836D83692F782F34
:1021E000902F812F8601C92ED82E1601201A310A70
:1021F0002B012D813E81421A530A57FE03C0519490
:1022000041945108710137FE03C03FEFE31AF30A0E
:10221000F594E7948D819E81861797075CF5A1E080
:10222000B0E0BA83A983C016D1064CF1D301ED9179
:10223000FC910484F585E02D2B813C81A8016D8102
:102240007E818A149B041CF04D815E81B801C3011C
:102250000995E418F508F7FE0AC02D813E818981B1
:102260009A81280F391F3E832D83E20CF31C0F5FE8
:102270001F4FD9CF2FEF3FEF3A832983D4CF269634
:102280000FB6F894DEBF0FBECDBFDF91CF911F9187
:102290000F91FF90EF90DF90CF90BF90AF909F9005
:1022A0008F907F906F905F904F903F902F90089508
:1022B000089520911302260F3327331F2132310551
:1022C000ECF420913702FC0190E080E0243069F0CA
:1022D00082E00895A09113022191AC014D505E4F10
:1022E000A40FB52FB11D2C930196861798F38091FA
:1022F0001302680F6093130280E0089581E008954F
:102300001092370281E0809339021092380261E026
:1023100082E10E94000761E083E10E940007E9EB8F
:10232000F0E080818E7F808380818D7F808388E450
:102330008093B80085E48093BC000895CF93DF9329
:1023400091E09093F2018823B9F0C091B800D09148
:10235000BA008091BC008A7B8093BC0060E082E17F
:102360000E94000760E083E10E9400070E94801144
:10237000D093BA00C093B800DF91CF910895E09157
:10238000630280916202E81730F4F0E0E353FE4FFD
:10239000808190E008958FEF9FEF08959091630200
:1023A000809162022FEF3FEF981748F4E92FF0E099
:1023B000E353FE4F208130E09F5F90936302C90199
:1023C00008958091620290916302891B990B089590
:1023D000CF92DF92EF92FF920F931F93CF93DF93F1
:1023E0007C01CB018A0120918802222389F0EB0134
:1023F0006B01C40ED51ECC15DD0569F06991D701BE
:10240000ED91FC910190F081E02DC7010995F3CF8A
:10241000642F0E945911C801DF91CF911F910F9134
:10242000FF90EF90DF90CF900895CF93DF931F92AE
:10243000CDB7DEB76983209188022223F9F020917D
:102440008502203258F021E030E0FC013383228302
:1024500090E080E00F90DF91CF9108958091860207
:10246000E82FF0E0E355FE4F998190838F5F8093D2
:1024700086028093850281E090E0ECCF61E0CE019E
:1024800001960E945911F7CFCF92DF92EF92FF92FF
:102490000F931F93CF93DF93D091850281E0D132C8
:1024A00008F09CC0C09187020E946A076B017C0102
:1024B0008091370281116CC082E08093370281E005
:1024C000809339028FEF8093360210925B02D09393
:1024D0005A02ADEAB1E0EAE3F2E080E0D8138DC041
:1024E00010925C0280915C02CC0FC82BC0935C02FE
:1024F00080913802813009F084C0109238020E9425
:102500006A076B017C0180915C028093BB00809123
:10251000EE019091EF01A091F001B091F101892BB2
:102520008A2B8B2BA1F00E946A070091EE0110917B
:10253000EF012091F0013091F1016C197D098E09B4
:102540009F09061717072807390708F442C080912A
:10255000BC0083FDD8CF85EC8093BC000E946A0745
:102560006B017C0180913702823009F44CC080916C
:1025700036028F3F09F469C080913602803209F437
:1025800066C080913602803309F463C084E026C0BF
:102590008091EE019091EF01A091F001B091F101D5
:1025A000892B8A2B8B2B09F483CF0E946A07009119
:1025B000EE011091EF012091F0013091F1016C19C1
:1025C0007D098E099F09061717072807390708F0A4
:1025D0006FCF8091ED010E949E1185E010928602DE
:1025E0001092850210928802DF91CF911F910F9176
:1025F000FF90EF90DF90CF9008959D9191938F5F22
:102600006DCF85EEA9CF8091EE019091EF01A09161
:10261000F001B091F101892B8A2B8B2B09F4A2CF09
:102620000E946A070091EE011091EF012091F001E4
:102630003091F1016C197D098E099F090617170762
:102640002807390708F08ECFC4CF80E0C7CF82E0DB
:10265000C5CF83E0C3CFEF92FF920F931F93CF9329
:10266000DF937C01C62F8091F7049091F8040097C6
:1026700009F459C02091FB0431E030938802209383
:1026800087021092860210928502DC01ED91FC9186
:102690000190F081E02D60E009958701EE24E3943C
:1026A000F12CD1E0C1508091F7049091F804CF3F14
:1026B00091F1B0E2EB16F104D8F00E94441280913F
:1026C000F7049091F8042091FB04D09388022093A2
:1026D00087021092860210928502DC01ED91FC9136
:1026E0000190F081E02D60E00995EE24E394F12C57
:1026F0008091F7049091F804F8016491DC01ED9168
:10270000FC910190F081E02D0995BFEFEB1AFB0AD7
:102710000F5F1F4FC7CFDF91CF911F910F91FF9098
:10272000EF900C944412E0910705F0910805908118
:1027300080910D058095892380838701C15008F41D
:1027400038C0F80184912091F5043091F604232BD0
:1027500029F00E94590B0F5F1F4FF0CF28E030E0A7
:1027600040E8E0910305F091040590910B05582F86
:102770005423D9F05081952B9083E0910505F09179
:102780000605908150910C05952B9083E0910505ED
:10279000F0910605508190910C05909595239083BA
:1027A000469521503109E9F6D6CF50819095952371
:1027B000E3CFDF91CF911F910F91FF90EF9008959C
:1027C0001F93CF93DF93EC018D8D9E8D009721F1A8
:1027D000162F29A131E030938802209387021092AE
:1027E000860210928502DC01ED91FC910190F0814E
:1027F000E02D60E009958D8D9E8DDC01ED91FC91C1
:102800000190F081E02D612F09958D8D9E8DDF91D6
:10281000CF911F910C944412ADA5BEA59C918BA99C
:10282000809589238C938B8D9C8D892B31F0862FFD
:10283000DF91CF911F910C94590B28E030E080E894
:10284000A9A5BAA599A9462F4823C1F04C91942B6C
:102850009C93ABA5BCA59C914AA9942B9C93ABA53A
:10286000BCA54C919AA9909594239C938695215050
:10287000310931F7DF91CF911F9108954C919095D7
:102880009423E6CFDF92EF92FF920F931F93CF93A3
:10289000DF938091F7049091F804892B09F4A5C087
:1028A00020910F05309110054091110550911205AE
:1028B00060E074E284EF90E00E94592920513109D0
:1028C0004109510956954795379527952093B800AA
:1028D00064E08BEC9CE00E942B138091DE049091CD
:1028E000DF048034910509F097C060E28AED94E03E
:1028F0000E94E0136091DE04615E8AED94E00E9424
:10290000E0132091E0043091E104C901079697FD9E
:10291000079633E0959587953A95E1F72091DE0487
:102920003091DF04829F8001839F100D929F100DD4
:102930001124C091F904D091FA048091F704909188
:10294000F8040C0F1D1F009709F498C02091FB0498
:1029500031E0309388022093870210928602109211
:102960008502DC01ED91FC910190F081E02D60E4A5
:102970000995EE24E394F12CDD24D3948091F7049F
:102980009091F8040C171D0709F44FC0B0E2EB1644
:10299000F104D8F00E9444128091F7049091F80459
:1029A0002091FB04D0928802209387021092860225
:1029B00010928502DC01ED91FC910190F081E02DF7
:1029C00060E40995EE24E394F12C8091F704909152
:1029D000F8046991DC01ED91FC910190F081E02D0A
:1029E0000995BFEFEB1AFB0AC9CF8091F5049091CE
:1029F000F604892B31F080911805909119050E94F9
:102A0000600BE0910905F0910A05908180910E0517
:102A10008095892380835CCF60E08AED94E00E94FA
:102A2000E0136091DE04615068CF0E9444128091EF
:102A3000F7049091F804892B09F461C020911305E3
:102A400030911405409115055091160560E074E22F
:102A500084EF90E00E945929205131094109510920
:102A600056954795379527952093B800DF91CF91DC
:102A70001F910F91FF90EF90DF900895E09107056F
:102A8000F0910805808190910D05892B80830C17AA
:102A90001D0769F289912091F5043091F604232BEA
:102AA00019F00E94590BF3CF28E030E040E8E091A4
:102AB0000305F091040590910B05582F5423D9F08C
:102AC0005081952B9083E0910505F091060590814A
:102AD00050910C05952B9083E0910505F09106052A
:102AE000508190910C0590959523908346952150A7
:102AF0003109E9F6CCCF508190959523E3CFE09151
:102B00000905F0910A05808190910E05892B80833B
:102B1000ADCF1F93CF93DF93EC01162F8D8D9E8D3C
:102B2000892BB1F12DA93EA94FA958AD60E074E2FF
:102B300084EF90E00E94592920513109410951093F
:102B400056954795379527952093B80066EA111159
:102B500067EACE010E94E0138D8D9E8D892B41F195
:102B600029AD3AAD4BAD5CAD60E074E284EF90E02E
:102B70000E9459292051310941095109569547951B
:102B8000379527952093B800DF91CF911F91089535
:102B90008B8D9C8D892B21F08EAD9FAD0E94600B9B
:102BA000EFA5F8A990818CA9809589238083CECF49
:102BB000EFA5F8A980819CA9892B8083E5CF90E0BF
:102BC00080E00895FC01848195812281338128175A
:102BD000390771F0860F971F608171810E947B29F0
:102BE0000680F781E02DE80FF91F808190E00895BD
:102BF0008FEF9FEF0895FC018481958122813381BD
:102C00002817390741F0860F971F608171810E9454
:102C10007B29958384830895FC01462F228133818B
:102C2000C9010196608171810E947B29648175814F
:102C30008617970781F0A681B781A20FB31F4C9327
:102C4000828193810196608171810E947B299383A7
:102C5000828380E008958FEF0895EF92FF920F93A3
:102C60001F93CF93DF937C01062F10E0B80182E21F
:102C700095E00E940C16D0E0C0E0C017D10758F4D0
:102C8000F701EC0FFD1F649170E082E295E00E9475
:102C90000C162196F2CFDF91CF911F910F91FF90EB
:102CA000EF900895CF93DF93FC01C281D38184819B
:102CB0009581C817D907C9F0A681B781A80FB91F98
:102CC0002C910196608171810E947B29C817D907D8
:102CD00039F095838483822F90E0DF91CF9108951E
:102CE0001582148213821282F6CF8FEF9FEFF5CFF9
:102CF000FC0160817181848195819B01281B390BC6
:102D000082819381820F931F0E947B290895DC01A9
:102D1000ED91FC910190F081E02D09948091AC013E
:102D20008823B9F08091AB01882399F06CE088E2A8
:102D300092E00E942D1667E081E292E00E942D163B
:102D400067E08AE192E00E942D1661E08AE00C942F
:102D5000000760E08AE00E94000767E084E392E0F9
:102D60000C942D168F929F92AF92BF92CF92DF92CA
:102D7000EF92FF924B015C010E946A076B017C019C
:102D800024E0C21AD108E108F1080E946A076C1910
:102D90007D098E099F09681579058A059B05A8F3A9
:102DA000FF90EF90DF90CF90BF90AF909F908F906B
:102DB000089580914E048F3F11F42D98089560E09E
:102DC0000C940007882349F080914E048F3F11F442
:102DD0002D9A089561E00C9400070C94D916CF93B6
:102DE000DF93EB0181E00E94E2162998BE0190E09A
:102DF00080E00E94B216299A0E94D916DF91CF91E5
:102E00000C94D9168F929F92AF92BF92CF92DF927D
:102E1000EF92FF921F93CF93DF93EC014A015B0186
:102E2000219A8FEF88169806A806B806E1F4219A31
:102E300060E073E2CE010E94EF1660EC78E080E083
:102E400090E00E94B21660E372E0CE01DF91CF9174
:102E50001F91FF90EF90DF90CF90BF90AF909F9029
:102E60008F900C94EF1660E073E2CE010E94EF1693
:102E700060E871E180E090E00E94B21610E2C12C9F
:102E8000D12CE12C90E8F92ED501C4018C219D2193
:102E9000AE21BF2160E372E0892B8A2B8B2B81F05E
:102EA000CE010E94EF1660E976E080E090E00E949B
:102EB000B216F694E794D794C794115029F7C3CF6C
:102EC000CE010E94EF1660E372E080E090E0EFCF69
:102ED0002091E0043091E104C901079697FD07961F
:102EE00023E0959587952A95E1F72091DE043091AE
:102EF000DF04829FA001839F500D929F500D1124EB
:102F000070E060E08091F9049091FA040C94C82A72
:102F1000FB0101900020E9F73197AF01461B570BE9
:102F2000DC01ED91FC910280F381E02D09948F92F8
:102F30009F92AF92BF920F931F93CF93DF93CDB722
:102F4000DEB7A1970FB6F894DEBF0FBECDBF19A2B2
:102F5000423008F44AE08E010F5D1F4F842E912C01
:102F6000B12CA12CA50194010E945929E62FB90189
:102F7000CA01EA3004F5E05DD801EE938D01232B00
:102F8000242B252B79F790E080E0109729F0BD01E4
:102F90008AED94E00E948817A1960FB6F894DEBFE0
:102FA0000FBECDBFDF91CF911F910F91BF90AF901A
:102FB0009F908F900895E95CDFCFCF93DF93682FC8
:102FC00070E090E080E04AE00E949717EC016EE923
:102FD00071E08AED94E00E9488178C0F9D1FDF91AD
:102FE000CF9108950F931F93CF93DF93EC010E942D
:102FF000D1078C016EE971E0CE010E948817800F25
:10300000911FDF91CF911F910F910895CF932AE9DE
:1030100034E0F90101900020E9F79F012B59344079
:10302000C091950433274C2F50E0BA0161507109CB
:10303000261B370B3093900420938F04682F70E089
:1030400066567B4F86E191E00E94BF2A809116016F
:10305000803219F486E880931601CB5FC09311018A
:10306000EC2FF0E0319620E090E0A92FB0E0A05FD7
:10307000BE4F4C9124279F5FC917B8F7E05FFE4F02
:1030800020836091110170E06E5F7F4F8AE295E0CE
:103090000E940C16C0E02C2F30E08091110190E0CE
:1030A0000196821793075CF0205F3E4FF901608123
:1030B00070E08AE295E00E940C16CF5FECCFCF91D2
:1030C00008950E94BA2A85ED8093BC008091EE019C
:1030D0009091EF01A091F001B091F1010796A11D2F
:1030E000B11D23E0B695A795979587952A95D1F7B9
:1030F0002091BC0024FD03C0109237020895409136
:10310000EE015091EF016091F0017091F101452BBA
:10311000462B472B69F30097A105B10541F02AE240
:103120002A95F1F700C00197A109B109E1CF80917B
:10313000ED010C949E111F93CF93DF93EC01162F9A
:103140000E944329181739F0612FCE01DF91CF91EA
:103150001F910C944B29DF91CF911F9108950C94EE
:1031600043298BE090E00E94AF18282F30E0309385
:10317000090120930801823071F018F4813031F098
:103180000895833061F0843071F008956AE182EB34
:1031900091E00C942D166AE180E092E0FACF6AE1AA
:1031A00086EE91E0F6CF6AE18CEC91E0F2CFCF931E
:1031B000DF9390E080E00E94AF18C82FD0E0D0935A
:1031C0000701C09306018AE090E00E94AF18282F03
:1031D00030E03093050120930401C130D10559F44A
:1031E000823011F1833021F1813029F46AE182EBE0
:1031F00091E00E942D168AE090E00E94AF18282FDF
:1032000030E030930501209304012297E9F48230E5
:1032100099F08330A9F08130B9F46AE188E991E04E
:10322000DF91CF910C942D166AE180E092E0E1CF1E
:103230006AE186EE91E0DDCF6AE18EE791E0F0CFC2
:103240006AE184E691E0ECCFDF91CF91089590E0C0
:1032500080E00E94AF18282F30E0309303012093C4
:1032600002018150873008F047C0E82FF0E0E55CAC
:10327000F64E0C948F294219481953195C19651997
:10328000691972191092AB010E948E160C94B11834
:103290001092AB010E948E166AE188E991E00E94CB
:1032A0002D160C94D7181092AB010E948E166AE16D
:1032B0008AE491E00C942D166AE180E391E00E948B
:1032C0002D161092AB010C948E166AE186E191E006
:1032D000F6CF6AE18CEF90E00E942D1681E080939A
:1032E000AB01F1CF1092AB010E948E166AE182EE23
:1032F00090E00E942D16E7CF08954F925F926F9253
:103300007F92AF92BF92CF92DF92EF92FF920F9394
:103310001F93CF93DF93CDB7DEB768970FB6F894BE
:10332000DEBF0FBECDBF7C01FC01D080A280C38078
:103330000481B58016810E94C1074090A20150907F
:10334000A3016090A4017090A5019B01AC01241918
:1033500035094609570929013A0130E1431637E298
:1033600053066104710468F06093A2017093A30195
:103370008093A4019093A50165E088E690E00E9407
:103380002D1645E050E06DED70E0C7010E94362932
:10339000892B29F466E087ED90E00E942D1646E027
:1033A00050E061ED70E0C7010E943629892B19F4C5
:1033B00081E08093AC0180917B0281110AC066E0BC
:1033C0008DE99CE00E942D160E94271981E08093D0
:1033D0007B0245E050E06CEC70E0C7010E943629AA
:1033E000892B29F466E086EC90E00E942D1645E0DA
:1033F00050E060EC70E0C7010E943629892B11F47F
:103400000E94271940E8D412E7C25FEBA512E7C279
:1034100088E1C812E4C2B0926D02802F90E0880F5C
:10342000991F90936F0280936E0245E0489F900130
:10343000499F300D11242C5F3F4F43E0369527956F
:103440004A95E1F730937502209374024FE0429F52
:10345000C001439F900D1124839666E470E00E94A2
:103460007B29615F7F4F6432710510F063E270E089
:1034700060930F0111E010937A0261E081E10E94F4
:1034800000078091AA01811104C00E94271910939E
:10349000AA0168960FB6F894DEBF0FBECDBFDF91CC
:1034A000CF911F910F91FF90EF90DF90CF90BF9041
:1034B000AF907F906F905F904F900895153009F412
:1034C000D8C0163031F766E08AE990E00E942D16E8
:1034D0008091AB01882309F414C18091AC01882349
:1034E00009F40FC167E083E990E0EAC01A3009F4FB
:1034F00087C108F042C0183009F408C1193049F6F4
:1035000090E080E00E94AF1890E0909307018093D4
:103510000601019709F035C14FE450EB62E67DE901
:1035200085E692E00E9402178091080190910901BE
:103530000196843091050CF021C19093090180938C
:103540000801609108018BE090E00E949B1868964A
:103550000FB6F894DEBF0FBECDBFDF91CF911F91A4
:103560000F91FF90EF90DF90CF90BF90AF907F9042
:103570006F905F904F900C94B1181B3009F481C18B
:103580001C3009F086CF66E087E890E00E942D1697
:1035900047E158EE62E67DE93FC21A3209F4A1C163
:1035A000F8F4173209F4EAC180F4163209F071CF49
:1035B0008091AB01882321F08091AC01811182C000
:1035C0004FE650E962E67DE927C2183209F4E3C10B
:1035D0004FE950E662E67DE9193209F41DC259CF80
:1035E0001D3209F4A5C158F41B3209F49CC14FE304
:1035F00050EC62E67DE91C3209F40EC24ACF1E325D
:1036000009F4B7C11E3409F044CF60E08AE068963F
:103610000FB6F894DEBF0FBECDBFDF91CF911F91E3
:103620000F91FF90EF90DF90CF90BF90AF907F9081
:103630006F905F904F900C94000766E08AEB90E0EB
:103640000E942D1647ED58E262E67DE985E692E09C
:103650000E94021780917202882339F080910E0136
:10366000833218F48F5F80930E0181E080937A0299
:1036700010CF66E084EB90E00E942D1647E558EAF3
:1036800062E67DE985E692E00E940217809172026F
:10369000882359F380910E01882339F38150E3CFB9
:1036A00066E08EEA90E00E942D168091AB0167E003
:1036B0008823F1F08091AC018823D1F087EA90E073
:1036C0000E942D1668960FB6F894DEBF0FBECDBFD0
:1036D000DF91CF911F910F91FF90EF90DF90CF90EE
:1036E000BF90AF907F906F905F904F900C948E162C
:1036F00080EA90E00E942D164FE250ED62E67DE9EF
:103700008BC14FEA50E562E67DE986C166E08DE84F
:1037100090E00E942D1647EC58E362E67DE985E6CD
:1037200092E00E940217809102019091030101969C
:103730008830910504F59093030180930201609114
:10374000020190E080E00E949B1868960FB6F89402
:10375000DEBF0FBECDBFDF91CF911F910F91FF90C4
:10376000EF90DF90CF90BF90AF907F906F905F9081
:103770004F900C94271981E090E0DDCF81E090E03C
:10378000DCCE90E080E00E94AF1890E090930701BB
:1037900080930601029709F07CCE4FE450EB62E67D
:1037A0007DE985E692E00E940217809104019091E4
:1037B000050101968430910504F5909305018093ED
:1037C0000401609104018AE090E00E949B186896D1
:1037D0000FB6F894DEBF0FBECDBFDF91CF911F9122
:1037E0000F91FF90EF90DF90CF90BF90AF907F90C0
:1037F0006F905F904F900C94D71881E090E0DDCFF0
:103800008091000190910101019686309105A4F507
:103810009093010180930001609100018CE890E099
:103820000E949B188CE890E00E94AF1890E0909363
:1038300001018093000128E1E6E3F1E0DE01119649
:1038400001900D922A95E1F7880F991F880F991F13
:10385000E1E0F0E0EC0FFD1F8E0F9F1FFC014081A7
:1038600051816281738186EA91E00E9402174FECD8
:1038700050E362E67DE9D0C0109201011092000190
:10388000CBCF4EE251ED62E67DE9C6C061E08AE051
:103890000E9400078CE00E94D706892B29F060E087
:1038A0008CE00E94000751CF61E08CE00E9400078D
:1038B0006AE18DE690E068960FB6F894DEBF0FBE21
:1038C000CDBFDF91CF911F910F91FF90EF90DF90CF
:1038D000CF90BF90AF907F906F905F904F900C947F
:1038E0002D168091730291E08927809373028823BB
:1038F00099F01092720283E2809371028FE08093BC
:1039000070020E94C1076093690270936A028093FB
:103910006B0290936C02A9CE109272021092710207
:1039200010927002A2CE46EB59E462E67DE974C0C3
:1039300061E090E080E00E949B1861E08AE090E006
:103940000E949B1861E08BE090E00E949B1860E071
:103950008EE190E00E949B1860E088E290E00E9477
:103960009B1860E08CE890E00E949B180E94271949
:103970002ECF4FE550EA62E67DE94EC08091AB0163
:10398000882321F08091AC0181119CCE4FE150EE53
:1039900062E67DE941C04FEE50E162E67DE985E6F1
:1039A00092E00E94021762E090E080E068960FB615
:1039B000F894DEBF0FBECDBFDF91CF911F910F9165
:1039C000FF90EF90DF90CF90BF90AF907F906F907F
:1039D0005F904F900C949B1820ECD2125ACDF1E3DB
:1039E000CF1257CD61E085E00E9400071E3009F438
:1039F0004DCF08F0D2CD173009F452CE08F076CD75
:103A0000143009F41ACE08F059CD47E958E662E6B9
:103A10007DE9133009F03DCD85E692E068960FB65A
:103A2000F894DEBF0FBECDBFDF91CF911F910F91F4
:103A3000FF90EF90DF90CF90BF90AF907F906F900E
:103A40005F904F900C9402171F920F920FB60F9237
:103A500011242F933F938F939F93AF93BF938091A4
:103A60007D0290917E02A0917F02B0918002309100
:103A70007C0223E0230F2D3758F50196A11DB11DBF
:103A800020937C0280937D0290937E02A0937F021C
:103A9000B09380028091810290918202A091830272
:103AA000B09184020196A11DB11D80938102909373
:103AB0008202A0938302B0938402BF91AF919F9141
:103AC0008F913F912F910F900FBE0F901F901895DF
:103AD00026E8230F0296A11DB11DD2CF1F920F928F
:103AE0000FB60F9211242F933F934F935F936F93D1
:103AF0007F938F939F93AF93BF93EF93FF93E09147
:103B00000C01F0910D010995FF91EF91BF91AF91DB
:103B10009F918F917F916F915F914F913F912F91E5
:103B20000F900FBE0F901F9018951F920F920FB617
:103B30000F9211242F933F934F935F936F937F9333
:103B40008F939F93AF93BF93EF93FF93E0910A01FD
:103B5000F0910B010995FF91EF91BF91AF919F916A
:103B60008F917F916F915F914F913F912F910F9026
:103B70000FBE0F901F9018951F920F920FB60F92C5
:103B800011242F933F934F935F936F937F938F9362
:103B90009F93AF93BF93EF93FF9389E892E00E94C6
:103BA0007308FF91EF91BF91AF919F918F917F919A
:103BB0006F915F914F913F912F910F900FBE0F909A
:103BC0001F9018951F920F920FB60F9211242F93EA
:103BD0008F939F93EF93FF93E0919902F0919A0254
:103BE0008081E0919F02F091A00282FD1BC0908134
:103BF0008091A2028F5F8F732091A302821741F000
:103C0000E091A202F0E0E757FD4F958F8093A2026A
:103C1000FF91EF919F918F912F910F900FBE0F9079
:103C20001F9018958081F4CF1F920F920FB60F92BC
:103C300011242F933F934F935F936F937F938F93B1
:103C40009F93AF93BF93EF93FF938091B900887FC9
:103C5000803609F44AC0F0F5883209F4A7C018F597
:103C6000803109F49BC0B8F4882309F4F9C0883086
:103C700009F494C0FF91EF91BF91AF919F918F9103
:103C80007F916F915F914F913F912F910F900FBE58
:103C90000F901F901895883109F488C0803251F731
:103CA0008093360214C0803409F49DC040F4803300
:103CB000B9F38833F9F68093360285ECB0C08035CD
:103CC00009F485C0883509F496C0883499F60E94B5
:103CD0006318D0CF883909F48CC038F5883729F0BB
:103CE00050F4883611F0803729F683E0809337024C
:103CF0001092350257C0883809F47BC0803919F01A
:103D0000803809F0B7CF80913502803208F071C059
:103D1000E091350281E08E0F809335028091BB00E7
:103D2000F0E0EB5EFD4F80833DC0803B39F0E0F476
:103D3000803A09F479C0883A09F09CCF84E08093F6
:103D400037021092140210921302E0916002F09177
:103D5000610209958091130281110FC081E0809367
:103D600013021092F30109C0803C09F4A6CF883CED
:103D700009F4A3CF883B09F07DCFE091140281E0E4
:103D80008E0F80931402F0E0ED50FE4F80818093FF
:103D9000BB00909114028091130229C080915C02B3
:103DA0008093BB0085EC8093BC0064CF90915B0254
:103DB00080915A02981758F5E0915B0281E08E0FCE
:103DC00080935B02F0E0E65CFD4F8081E9CFE091FB
:103DD0005B0281E08E0F80935B028091BB00F0E07C
:103DE000E65CFD4F808390915B0280915A029817A8
:103DF000C8F285E8D8CFE0915B0281E08E0F809316
:103E00005B028091BB00F0E0E65CFD4F8083809117
:103E1000390281115CCF81E08093380284EA80937B
:103E2000BC001092370226CF85EC8093BC00109224
:103E3000370280913502803230F4E0913502F0E0B3
:103E4000EB5EFD4F10826091350270E0E0915E0202
:103E5000F0915F0285E192E00995109235020ACF58
:103E60001092360234CF1F920F920FB60F92112488
:103E70002F933F934F935F936F937F938F939F9372
:103E8000AF93BF93EF93FF9381E08093640260E070
:103E90008DE00E940007E1EBF0E08081887F808365
:103EA000FF91EF91BF91AF919F918F917F916F9112
:103EB0005F914F913F912F910F900FBE0F901F90E8
:103EC00018951F920F920FB60F9211242F933F93C4
:103ED0004F935F936F937F938F939F93AF93BF9312
:103EE000EF93FF9380E00E94D7060197D9F481E019
:103EF0000E94D7060197B1F48091B100876080934A
:103F0000B100FF91EF91BF91AF919F918F917F9100
:103F10006F915F914F913F912F910F900FBE0F9036
:103F20001F90189580E00E94D706892B51F781E0F9
:103F30000E94D706019729F71092640261E08DE094
:103F40000E9400078091B100887FD9CF1F920F9205
:103F50000FB60F9211242F933F934F935F936F935C
:103F60007F938F939F93AF93BF93CF93EF93FF93E1
:103F7000E0913C03F0913D03C08180913E03C82352
:103F800080913F039091400320913F033091400383
:103F90002F3F3F4F29F001969093400380933F03BA
:103FA00020913A03211115C0C1114BC0813A9105EE
:103FB00058F01092490390934C0380934B0381E097
:103FC00080934A0380933A031092400310923F0378
:103FD00038C0213099F4CC23A1F1E0914A032E0F8F
:103FE00020934A03F0E0E65CFC4F8F3F910519F007
:103FF00010F08FEF90E0838B82E0E4CF223009F065
:1040000047C0E0914A03813A910510F4E73CA0F1E2
:10401000E83C18F081E08093490380914B03909134
:104020004C039093420480934104E093400483E066
:1040300080933A03E0914103F0914203309709F0F5
:10404000099580914F04882329F081E0C11180E017
:104050000E94E216FF91EF91CF91BF91AF919F9196
:104060008F917F916F915F914F913F912F910F9021
:104070000FBE0F901F901895C111E3CF91E09E0FD6
:1040800090934A03F0E0E65CFC4F838B81E09ACF8B
:104090002330B9F6C111D5CF97CFFC018681978126
:1040A000009711F00C94312A089586E791E09093DF
:1040B000DB048093DA048091F9049091FA0400976C
:1040C00011F00E94312A8AE295E00E944D2082E29E
:1040D00095E00E944D208AE195E00C944D200F93CD
:1040E0001F93CF93DF93EC018B01798368831D824B
:1040F0001C821B821A82CB010E9495299F838E838A
:10410000A80170E060E0DF91CF911F910F910C94B6
:10411000C82AEF92FF920F931F93CF93DF93E9E8A2
:10412000F2E01382128288EE93E0A0E0B0E0848394
:104130009583A683B78322E531E03183208325EC84
:1041400030E03587248724EC30E03787268720EC61
:1041500030E0318B208B21EC30E0338B228B22EC52
:1041600030E0358B248B26EC30E0378B268B118E9C
:10417000128E138E148E2EE2E22E23E0F22EF70121
:104180001382128284839583A683B78384E691E0A9
:10419000918380830E94C10760932A0370932B034D
:1041A00080932C0390932D030E94C10760932603F4
:1041B00070932703809328039093290360E870E0AD
:1041C0008AE195E00E946F2060E470E082E295E071
:1041D0000E946F2060E470E08AE295E00E946F2008
:1041E0001FEF10934E04EAE3F3E0118201E0048331
:1041F00089E290E0938382835098C0E5D4E01CAAC2
:104200000E94C10760932A0370932B0380932C03B1
:1042100090932D030E94C107609326037093270398
:10422000809328039093290319861A861B86188683
:104230001F821E821D8262E080E00E942E0761E0E4
:1042400084E00E942E0761E084E00E940007E0EB1A
:10425000F0E010821092B1008DE98093B30080816C
:1042600082608083E0E7F0E0808182608083E8E61E
:10427000F0E0808184608083EDE6F0E08081816001
:10428000808319821A8280ED97E09AAF89AF88EE19
:1042900093E09CAF8BAF88EC90E09EAF8DAF82E057
:1042A000809396041092900410928F048BE0809378
:1042B00095041092970410929804109299040E9409
:1042C000C107609391047093920480939304909338
:1042D0009404EAEDF4E01382128220E830E03583A2
:1042E000248380E290E097838683318720879387B9
:1042F0008287168A1586148617861686058B048B88
:104300008FEF9FEF938B828B918B808B078B108E1F
:10431000128E118E86E791E091838083148E138E26
:10432000F68EE58E10A2178E14A315A316A317A35D
:1043300010A780E89AE1A6E0B0E085AB96ABA7AB0A
:10434000B0AF80EA96E8A1E0B0E081AF92AFA3AF52
:10435000B4AF80E586AF17AEDF91CF911F910F917B
:10436000FF90EF900895789484B5826084BD84B501
:10437000816084BD85B5826085BD85B5816085BD60
:1043800080916E00816080936E0010928100809118
:1043900081008260809381008091810081608093A0
:1043A0008100809180008160809380008091B100C5
:1043B00084608093B1008091B00081608093B000F0
:1043C00080917A00846080937A0080917A00826084
:1043D00080937A0080917A00816080937A00809146
:1043E0007A00806880937A001092C1001092630274
:1043F0001092620210928602109285020E94801131
:104400008EEC97E090936102809360028FEC97E0CE
:1044100090935F0280935E0268EC70E080E090E031
:104420000E948F078091F9049091FA04892B41F53D
:104430002091E0043091E104C901079697FD0796A9
:10444000B3E095958795BA95E1F72091DE04309118
:10445000DF04AC01429FC001439F900D529F900D1D
:1044600011240E9495299093FA048093F904892BD2
:1044700039F46BE27CE089E892E00E94F217FFCF0A
:104480000E9468172091E0043091E1048091DE04DD
:104490009091DF04B901213231050CF423C260543C
:1044A000710977FF02C06F5F7F4F759567958255E1
:1044B000910997FD019600E410E022E530E04DE31C
:1044C00059E0959587950E944A1082E08093FC04FC
:1044D0008091F7049091F804892B09F416C28CE3BB
:1044E0008093FB0410926302109262021092860283
:1044F000109285020E9480118EEC97E090936102E9
:10450000809360028FEC97E090935F0280935E024D
:104510008091020587FD1EC061E00E942E0761E0C8
:10452000809102050E94000761E070E080E090E069
:104530000E948F0760E0809102050E9400076AE0F8
:1045400070E080E090E00E948F0761E080910205BA
:104550000E9400078091F7049091F804892B09F4D8
:1045600093C220910F053091100540911105509193
:10457000120560E074E284EF90E00E945929205116
:10458000310941095109569547953795279520934B
:10459000B80064E089E597E00E942B136091E00485
:1045A00061508AED94E00E94E01364E085E597E0B5
:1045B0000E942B138091FC0460E1813009F064E1DA
:1045C0008AED94E00E94E01364E081E597E00E94A8
:1045D0002B138FE8809317058091DE049091DF0400
:1045E0008038910509F067C28091E0049091E10460
:1045F0008034910509F06FC28091FC04813009F08C
:104600007DC28FE980931705C2E16AED8AED94E0DF
:104610000E94E0136C2F8AED94E00E94E01361E8A1
:104620008AED94E00E94E013609117058AED94E012
:104630000E94E01369ED8AED94E00E94E0138091FE
:10464000FC0462E2813009F061EF8AED94E00E949F
:10465000E01366E08BE497E00E942B138091F7044F
:104660009091F804892B09F44BC2209113053091E5
:104670001405409115055091160560E074E284EF31
:1046800090E00E945929205131094109510956955C
:104690004795379527952093B8000E946817C1E089
:1046A000C093EE04C093EF0481E090E09093ED049A
:1046B0008093EC049093EB048093EA041092E70457
:1046C0001092E6041092E9041092E804C093F204F8
:1046D00061E27CE08AED94E00E94F2176FE07CE0FA
:1046E0008AED94E00E94F2176DEF7BE08AED94E092
:1046F0000E94F2170E94421461E085E00E942E079A
:1047000061E086E00E942E0760E08AE00E942E07AA
:1047100061E08BE00E942E0761E08CE00E942E0792
:1047200062E084E10E942E0761E08DE00E942E0786
:10473000E0919902F0919A02D2E0D083E091950243
:10474000F09196021082E0919702F091980280E138
:1047500080831092A102E0919D02F0919E0286E07A
:104760008083E0919B02F0919C0280818061808334
:10477000E0919B02F0919C02808188608083E091AF
:104780009B02F0919C02808180688083E0919B0273
:10479000F0919C0280818F7D808361E085E00E94A2
:1047A0000007C09388028FE28093870210928602EE
:1047B000109285026FE78EE293E00E9415128EE25E
:1047C00093E00E94441289E892E09093540480930D
:1047D0005304E0919902F0919A02D083E0919502FE
:1047E000F09196021082E0919702F09198028FEC7E
:1047F00080831092A102E0919D02F0919E0286E2D8
:104800008083E0919B02F0919C0280818061808393
:10481000E0919B02F0919C02808188608083E0910E
:104820009B02F0919C02808180688083E0919B02D2
:10483000F0919C0280818F7D80838CED95E0909338
:104840008A048093890488EE93E090938C0480938B
:104850008B0488EC90E090938E0480938D04D09329
:1048600096048DE799E1909388048093870461E032
:104870008DE00E942E0722E0422E512C01E010E034
:1048800034E0632E712C43E0A42EB12CC1E090E003
:10489000292E90E0392E80917B0281110FC068EEA5
:1048A00073E080E090E00E948F0766E08DE99CE075
:1048B0000E942D160E942719C0937B02E091550497
:1048C000F0915604E830F10508F026C1E659FB4D99
:1048D0000C948F298A25622678269926C226D72607
:1048E000EB260C276052710977FF02C06F5F7F4F84
:1048F000759567958357910997FD019600E210E041
:1049000023E730E04DE557E0DCCD61E08091000524
:104910000E942E0761E0809101050E942E07809180
:104920000005082E000C990BFC01E752F34FE491AF
:10493000F0E0EE0FFF1FE355F34F259134913093D4
:10494000080520930705FC01E351F34FE491E09340
:104950000D0580910105082E000C990BFC01E75212
:10496000F34FE491F0E0EE0FFF1FE355F34FA591F5
:10497000B491B0930A05A0930905FC01E351F34FEC
:10498000E491E0930E058C91E82BEC938091F50473
:104990009091F604892B09F434C0CFB7F894809134
:1049A0005D02811127C0E3EEFCE08491E7EFFCE0BB
:1049B0009491E82FF0E0EE0FFF1FED55F34FA59116
:1049C000B491EC91E92321F461E08AE00E940007B0
:1049D00061E08AE00E942E078CB580618CBD8CB5A9
:1049E00080648CBD61E08DE00E942E0761E08BE069
:1049F0000E942E0780915D028F5F80935D02CFBF82
:104A000087CD61E08091FE040E942E0761E08091D5
:104A1000FF040E942E078091FE04082E000C990BC3
:104A2000FC01E752F34FE491F0E0EE0FFF1FE35576
:104A3000F34F259134913093040520930305FC0135
:104A4000E351F34FE491E0930B058091FF04082EAE
:104A5000000C990BFC01E752F34FE491F0E0EE0FEC
:104A6000FF1FE355F34FA591B491B0930605A093B2
:104A70000505FC01E351F34FE491E0930C058C91A3
:104A8000E095E823EC9344CD8091F5049091F604F1
:104A9000892B31F080911805909119050E94600BC7
:104AA000E0910905F0910A05908180910E058095AD
:104AB000892380836ECD8036910589F48091E0044E
:104AC0009091E104409739F48091FC04813029F4FD
:104AD00080E180931705C2E098CD8FEAFACF803449
:104AE0009105C9F78091E0049091E104809799F7CE
:104AF0008091FC04813011F480E184CD8FEC82CD73
:104B0000E0910905F0910A05808190910E05892BAD
:104B10008083C3CD10929704809164028823E9F0CA
:104B20008AE295E00E94781618161906B4F48AE213
:104B300095E00E9452166C0180E00E94D706019712
:104B400039F4F12CE12CF3E1CF16D10408F48AC139
:104B5000B6018AE295E00E94FB1580915304909182
:104B60005404DC01ED91FC910084F185E02D099560
:104B7000892B81F08091530490915404DC01ED91D4
:104B8000FC910284F385E02D0995BC018AE195E052
:104B90000E940C1680915704909158048230910520
:104BA00009F4B5C108F072C1009709F47DC10197FD
:104BB00009F48FC1809164028823D1F182E295E0EB
:104BC0000E947816181619069CF50E94C107C0901D
:104BD0002603D0902703E0902803F09029036C1956
:104BE0007D098E099F096A3071058105910500F1E3
:104BF00082E295E00E9452166C0180E00E94D70686
:104C0000019739F4F12CE12CB1E2CB16D1040CF46C
:104C100000C2B60182E295E00E94FB150E94C10726
:104C200060932603709327038093280390932903AE
:104C300080915104882371F00E94C10760E084E0F4
:104C40000E94000770E060E080915304909154044A
:104C50000E94871680917302882309F405C2C090D0
:104C60006902D0906A02E0906B02F0906C02809131
:104C700072028111ABC20E94C1076C197D098E09B5
:104C80009F09663971058105910508F4EDC1D09140
:104C90007102DD2309F4D1C147E558EA62E67DE9F6
:104CA00085E692E00E940217D150D09371020E94D3
:104CB000C1076093690270936A0280936B029093BC
:104CC0006C02D0C1109299041092980480E00E9466
:104CD000061850925604409255040E94C1076093F2
:104CE000910470939204809393049093940414CF4E
:104CF0000E94C107C0909104D0909204E090930468
:104D0000F0909404AB01BC014C195D096E097F0958
:104D10008091890490918A04B0E0A0E04817590777
:104D20006A077B0708F4F8CEB0925604A0925504A7
:104D3000F3CE2091980480918F04909190042817CD
:104D4000190680F42F5F209398048091990491E0D4
:104D5000980F909399040E940618709256046092DE
:104D60005504BBCF85E090E09093560480935504A2
:104D70001092990410929804809197048F5F809309
:104D80009704CACE0E94C107C0909104D0909204AB
:104D9000E0909304F0909404AB01BC014C195D09C0
:104DA0006E097F0980918D0490918E04B5CF90910A
:104DB000970480919604981738F4A6E0B0E0B09379
:104DC0005604A093550489CFE7E0F0E0F093560431
:104DD000E093550482CF0E94C107C0909104D09007
:104DE0009204E0909304F0909404AB01BC014C1940
:104DF0005D096E097F0980918B0490918C04B0E06D
:104E0000A0E0481759076A077B0708F485CE10937E
:104E100056040093550480CE0E94C107C0909104AF
:104E2000D0909204E0909304F0909404AB01BC0104
:104E30004C195D096E097F0980918B0490918C0457
:104E4000B0E0A0E0481759076A077B0708F464CE72
:104E50001092990480E00E94061810925604109255
:104E600055045ACE8090530490905404CE14DF041D
:104E700009F473CE8AE295E00E945216BC01C40187
:104E80000E9487162FEFE21AF20AECCF83309105C9
:104E900009F477C061E070E0049709F08BCE8AE1F5
:104EA00095E00E94FB15B0C08AE195E00E9478165B
:104EB000181619060CF07ECE70E060E08AE195E0ED
:104EC0000E94E215809359041093580400935704EC
:104ED00071CE8AE195E00E94781602970CF46ACEB2
:104EE00061E070E08AE195E00E94E21580935A0447
:104EF0008350823228F450925804409257045ACE7C
:104F000061E070E08AE195E00E94FB1553CEC0900D
:104F10005A04D12C4601BFEF8B1A9B0A8AE195E017
:104F20000E947816881699060CF044CED0E0F12C39
:104F3000E12CB7018AE195E00E94E215D827EFEF56
:104F4000EE1AFE0ACE14DF04A4F7B4018AE195E05C
:104F50000E94E215D817190679F40E94C1076093E0
:104F60002A0370932B0380932C0390932D03B0920C
:104F70005804A09257041ECE7092580460925704B1
:104F800019CE80915904982F9F77903521F0982F52
:104F90009F7B9038C9F480E5E82E84E0F82E9701D5
:104FA00020553440FFEFEF1AFF0A80915A0490E039
:104FB000019682179307FCF08AE195E00E94521651
:104FC000D7011B968C93EBCF893729F3982F9D7FC0
:104FD000983609F38F33F9F28831E9F2982F9F7DE3
:104FE000983CC9F260915A0470E06E5F7F4F803B3D
:104FF00009F055CFD0CFC0938404E0918704F0919D
:1050000088048CE594E00995109258041092570496
:10501000D1CDEC14FD040CF001CE8090530490909F
:10502000540482E295E00E945216BC01C4010E9421
:105030008716EFEFEE1AFE0AECCFD0917002DD2357
:1050400061F047ED58E262E67DE985E692E00E9474
:105050000217D150D09370022ACEFFE0F0930E01D8
:10506000C0937202C0937A0280917A02882309F475
:1050700091C00E94C107C0907602D0907702E09064
:105080007802F09079026C197D098E099F096436C7
:1050900071058105910508F47DC00E94C1076093E8
:1050A000760270937702809378029093790210923F
:1050B0007A020E946817C093EE04C093EF04109325
:1050C000ED040093EC041093EB040093EA041092B7
:1050D000E7041092E6041092E9041092E80465E9EE
:1050E0007CE08AED94E00E94D10760917402709197
:1050F000750290E080E04AE00E94971760E97CE04A
:105100008AED94E00E94F21767E87CE08AED94E073
:105110000E94D10760910F0170E090E080E04AE0CA
:105120000E9497178091730281117BC06BE77CE02E
:105130008AED94E00E94F21761E57CE08AED94E04C
:105140000E94D10760916E0270916F0290E080E042
:105150004AE00E9497176BE47CE08AED94E00E949D
:10516000F21765E47CE08AED94E00E94D10760913B
:105170006D0244E6649FB001112490E080E04AE0B3
:105180000E9497176EE971E08AED94E00E948817FB
:105190000E9442140E94C10761347F41810591053C
:1051A00048F08BE00E94D706019721F460E08BE085
:1051B0000E9400072114310409F46DCB0E945F089E
:1051C000882309F463CB0E94000060CB0E94C107D2
:1051D0006C197D098E099F096C327140810591051A
:1051E00008F442CFD0910E0180910F01D81760F4DE
:1051F00047ED58E262E67DE985E692E00E940217FB
:10520000DF5FD0930E0153CD8D1708F02DCF47E50A
:1052100058EA62E67DE985E692E00E940217D150E5
:10522000F0CF80917202811118C0809171028823A1
:1052300059F060E77CE08AED94E00E94D10780910C
:1052400071020E94DD1778CF65E67CE08AED94E07C
:105250000E94D10780917002F4CF6AE57CE08AED6C
:1052600094E00E94D10780910E01EBCFFB01DC019D
:1052700004C08D910590801921F441505040C8F729
:10528000881B990B0895F999FECF92BD81BDF89ABC
:10529000992780B50895262FF999FECF1FBA92BDA0
:1052A00081BD20BD0FB6F894FA9AF99A0FBE019607
:1052B0000895A1E21A2EAA1BBB1BFD010DC0AA1F57
:1052C000BB1FEE1FFF1FA217B307E407F50720F06F
:1052D000A21BB30BE40BF50B661F771F881F991FEA
:1052E0001A9469F760957095809590959B01AC0133
:1052F000BD01CF010895AA1BBB1B51E107C0AA1F26
:10530000BB1FA617B70710F0A61BB70B881F991F66
:105310005A95A9F780959095BC01CD010895EE0F9F
:10532000FF1F0590F491E02D09940F931F93CF93E5
:10533000DF938230910510F482E090E0E091340533
:10534000F091350530E020E0B0E0A0E0309799F42E
:105350002115310509F44AC0281B390B24303105C9
:10536000D8F58A819B816115710589F1FB019383D1
:105370008283FE0111C0408151810281138148174F
:105380005907E0F04817590799F4109761F0129601
:105390000C93129713961C933296CF01DF91CF9105
:1053A0001F910F9108950093340510933505F4CFA4
:1053B0002115310551F04217530738F0A901DB01DF
:1053C0009A01BD01DF01F801C1CFEF01F9CF909340
:1053D000350580933405CDCFFE01E20FF31F819395
:1053E00091932250310939832883D7CF20913205F8
:1053F00030913305232B41F4209132013091330158
:1054000030933305209332052091300130913101E2
:105410002115310541F42DB73EB74091340150912B
:105420003501241B350BE0913205F0913305E2176D
:10543000F307A0F42E1B3F0B2817390778F0AC01B7
:105440004E5F5F4F2417350748F04E0F5F1F509394
:10545000330540933205819391939FCFF0E0E0E0D4
:105460009CCFCF93DF930097E9F0FC013297138232
:105470001282A0913405B0913505ED0130E020E0B5
:105480001097A1F420813181820F931F2091320562
:10549000309133052817390709F061C0F0933305BF
:1054A000E0933205DF91CF910895EA01CE17DF072F
:1054B000E8F54A815B819E0141155105B1F7E9018B
:1054C000FB83EA8349915991C40FD51FEC17FD075F
:1054D00061F4808191810296840F951FE90199837F
:1054E0008883828193819B838A83F0E0E0E0129637
:1054F0008D919C9113970097B9F52D913C9111973F
:10550000CD010296820F931F209132053091330511
:105510002817390739F6309751F510923505109252
:105520003405B0933305A0933205BCCFD383C28337
:1055300040815181840F951FC817D90761F44E5FD0
:105540005F4F88819981480F591F518340838A8119
:105550009B81938382832115310509F0B0CFF093AD
:105560003505E09334059ECFFD01DC01C0CF1382E9
:105570001282D7CF81E090E0F8940C94CF2AFB01FF
:10558000DC0102C001900D9241505040D8F70895BF
:10559000DC0101C06D9341505040E0F7089516E0E2
:1055A000C2E8D6E004C0FE010E948F292196C338CC
:0855B000D107C9F7F894FFCF01
:1055B80001000100010001000100D007D0070F0F12
:1055C800C8008023423200000000000000000000F4
:1055D80000000000000000000000000000000000C3
:1055E8000000360580007F80629DBF40629D3FC0FD
:1055F800629DDF20629D5FA0629D9F60629D0000AA
:1056080000009508F5072208E20853083108450804
:10561800000000001512E811DF15AD06E111CE11EA
:10562800BF11000000009E0DF507DF155811A90AEB
:10563800AD0643101B1037102B10AB10AD06640BD2
:105648008915190A620A640F470FCF0E700E0D0AEA
:02565800000050
:00000001FF
